:02000000802E50
:03000B00021DDCF7
:0300230002024D89
:20002E00E1767581227508FF7509BF90A668E4F01236B380ED12001B80FBC82581C822C9E7
:20004E002581C97A0022D083D082CF2581F581CFC082C08322CF2581F581CF22FBE0CB22DD
:20006E00FCE0FBA3E0CC22FAE0F9A3E0CA2229F9E5F03AFA227C00CB30E7011CCB2275F0CE
:20008E000030E70215F022FDE493A3FEE493A3FF4E7009E493FE740193FF800BE493A3B547
:2000AE00050BE493B5F0068F838E82E473A380D8FEEBA4FD8EF0ECA4FCEB8EF0A4C5F02C0A
:2000CE002DC5F02211D88EF0ED22C002C001AAF0F97E007D007F11C3E933F9EA33FADF0821
:2000EE00F5F0E9D001D00222ED33FDEE33FEC3ED9BF5F0EE9C40E0ADF0FED380DBBB0001C4
:20010E0022C333C5F033C5F0DBF722BB000122C3C5F013C5F013DBF722240280022401C571
:20012E00F03400C5F022C394028003C39401C5F09400C5F0223139F4C5F0F4C5F02245F04F
:20014E0070220422319B4024801A319B401E7014801A319B400E7014800A319B500E8004F1
:20016E0031AF6008E4F5F02231AF60F8E4F5F0042231AF40F780ED31AF40F170E780ED318D
:20018E00AF40E170E780DD31AF50E180D7C39BC5F09C20E70720D207C345F02220D2F9D3D7
:2001AE0022C5F0C39C7003E5F09B2290A668E0A360EEE0FFA3E0A3CF2582F582EF3583F5F9
:2001CE008380EB7E00CF2508F582EE3509F583EF227E00CF2508F9EE3509FAEF227E00C590
:2001EE00082FC508C5093EC50922E4F50AA88108E4F608B880FB22E4F520D201D200D20333
:20020E00D205C2B4E4F50EF50DF50CF50BE4F512F511F510F50F74FFF513E588543FF588A7
:20022E00E589540FF5894420F5897450F598E5874480F58774FAF58BF58DD28ED2AC22C052
:20024E00E0C0D0C083C082309839E50DB4FA028030502E050DE50DB50E0280044002F50E38
:20026E0090A000C0E0E50B2582F582E43583F583D0E0E599F0050BE50BB4FA004003750BEF
:20028E0000C298309948E511700DD200300235E4D5E0FDC2B4802DC20030011A300202D26D
:2002AE00B490A0FAC0E0E5102582F582E43583F583D0E0E0F59915110510E510B4FA00404F
:2002CE0003751000C299200105200002D299D082D083D0D0D0E0322278FB120048E6C0E0DE
:2002EE00B40A0B300308D204740D1581C0E0E511B4FA0280F950F7C2AC90A0FAC0E0E50FCD
:20030E002582F582E43583F583D0E0D0E0C0E0F00511050FE511B512004002F512E50FB4D5
:20032E00FA004003750F00300002D299D2ACD0E0300408C204740AC0E080B322E4F5F0786D
:20034E00FB120048F608A6F022E51364FF7038E50D6034300531C2AC90A000C0E0E50C2541
:20036E0082F582E43583F583D0E0E0D2ACB40A0302038574018010150D050CE50CB4FA0032
:20038E004003750C0080C875F00022E4A20192E0F51F70030203BAE51160030203A5E4A2F4
:2003AE000092E0F51FE51F70030203AC22C2AC7513FF7400F50CF50BC50DD2AC75F000221E
:2003CE0074FFC513B4FF2EE50D0060FBC2AC90A000C0E0E50C2582F582E43583F583D0E085
:2003EE00E0C0E0150D050CE50CB4FA004003750C00D2ACD0E030050BB40A030203D5B40D0F
:20040E0002740A75F000221203CEC0E0C0E0C0E01202E6D0E0D0E0D0E075F00022E5137506
:20042E00F0007BFF7C0012016E700302044374FFF5F002045378FB120048E60886F0F513A1
:20044E0018E60886F02278FB1200488682088683E06016C083C082C0E0C0E01202E6D0E045
:20046E00D0E0D082D083A380E722E4F5F078FB120048F608A6F022746A75F03CC0E0C0F0D2
:20048E00E52075F000C0E0C0F074021237721581158115811581748575F03CC0E0C0F0E53C
:2004AE000F75F000C0E0C0F0E510C0E0C0F0E51175F000C0E0C0F0E512C0E0C0F074057545
:2004CE00F0001237727FF612005474B875F03CC0E0C0F0E50B75F000C0E0C0F0E50CC0E035
:2004EE00C0F0E50D75F000C0E0C0F0E50EC0E0C0F0740575F0001237727FF6120054E4F507
:20050E000EF512227FFD7EFF1201EDE4F5F07F001201D1F0A3C5F0F0C5F078FB120048E6D1
:20052E000886F012013918F608A6F012012B45F06022181818860108860289828A831200B9
:20054E007589828A83E012008CC0E0C0F012386B1581158145F0700302061E7F001201D120
:20056E00E0A3F5F0E0C5F07B047C0012010B7F001201D1F0A3C5F0F0C5F078F912004886B6
:20058E000108860289828A8312007589828A83E012008CC0E0C0F012387A158115817F02C6
:2005AE001201D1F07F021201D1E012008C7B39120083120158600B7F021201D1E0C394308B
:2005CE00800B7F021201D1E0C39441240A75F0007F001201D112006E2BC5F03CC5F07F00DF
:2005EE001201D1F0A3C5F0F0C5F078F9120048860108860289828A83E0A3F5F0E0C5F01213
:20060E00012B89828A83F0A3C5F0F0C5F00205287F001201D1E0A3F5F0E0C5F07F03020187
:20062E00EB7FF17EFF1201ED7F021201DFE98AF0C0E0C0F0E4C0E0C0E0740A75F000C0E007
:20064E00C0F01238AC7FFA1200547F021201DFE98AF07F0C1201D1F0A3C5F0F0C5F0740958
:20066E007F0E1201D1F078FB120048860108860289828A8312007589828A83E012008CC032
:20068E00E0C0F01238321581158145F0602E78FB120048860108860289828A831200758945
:2006AE00828A83E012008CC0E0C0F01238661581158145F060067F0E1201D1E0700302078B
:2006CE003E7F0C1201D1E0A3F5F0E0C5F012012B7F0C1201D1F0A3C5F0F0C5F0120139F983
:2006EE00AAF0C001C00278F9120048860108860289828A8312007589828A83E0D083D082B1
:20070E00F018860108860289828A83E0A3F5F0E0C5F012012B89828A83F0A3C5F0F0C5F054
:20072E007F0E1201D1E0147F0E1201D1F00206747F021201DFE98AF0C0E0C0F01238CF1515
:20074E008115817F001201D1F0A3C5F0F0C5F07F0F0201EB7FFE7EFF1201EDE4F5F07F0066
:20076E001201D1F0A3C5F0F0C5F07F001201D1E0A3F5F0E0C5F012014C45F0601B78FB12A6
:20078E000048E60886F012013918F608A6F012012B7B007C0012016045F0700302080878CD
:2007AE00F7120048E60886F012012B18F608A6F0120139F9AAF089828A83E012008CC0E077
:2007CE00C0F008E60886F012012B18F608A6F0120139F9AAF089828A83E012008CFBACF0F9
:2007EE00D0F0D0E0C39BC5F09CC5F07F001201D1F0A3C5F0F0C5F00207787F001201D1E003
:20080E00A3F5F0E0C5F07F020201EB7FFF7EFF1201EDE47F001201D1F07F001201D1E07554
:20082E00F0007B107C0012018570120208887F001201D1E0047F001201D1F080DC78FB128C
:20084E000048E60886F07F001201D112006A2BC5F03400C5F0F9AAF07F001201D1E0C0019F
:20086E00C00279567AA412008C12007C89828A83E0F4D083D082F002083C740190A47AF0B5
:20088E007F010201EB7FFF7EFF1201EDE4F521E4F5F090A2BEF0A3C5F0F0C5F0E490A2BD6E
:2008AE00F074F475F0A1C0E0C0F0E4C0E0C0E074C975F000C0E0C0F01238AC7FFA12005491
:2008CE00E4F5F090A389F0A3C5F0F0C5F074C075F0A2C0E0C0F0E4C0E0C0E074C975F00047
:2008EE00C0E0C0F01238AC7FFA120054E490A455F0748C75F0A3C0E0C0F0E4C0E0C0E07478
:20090E00C975F000C0E0C0F01238AC7FFA120054740190A47AF0E47F001201D1F07F00129B
:20092E0001D1E075F0007B107C0012017F70120209997F001201D1E0047F001201D1F080B9
:20094E00DC7F001201D1E079567AA412008C12007C7F001201D1E0C001C00279687AA4127A
:20096E00008C12007C89828A83E0F412008CD083D08212006A120083120176700302099672
:20098E00E490A47AF002099902094090A47AE060030209DE745675F0A4C0E0C0F0E4C0E057
:2009AE00C0E0741275F000C0E0C0F01238AC7FFA120054745675F0A4C0E0C0F0745F75F01E
:2009CE003CC0E0C0F0123918158115811581158112175B121808746875F0A4C0E0C0F012C5
:2009EE000819158115817F010201EB12039978FB120048E60886F090A38BF0C209C2B490D0
:200A0E00A38BE075F000900A37020095E490A38BF0D208C202E490A667F0020A4BC208D259
:200A2E0002E490A667F0020A4B2B0A03002B0A02002B0A01001F0A000000001A0A227FFB50
:200A4E007EFF1201ED78F9120048E60886F07F031201D1F0A3C5F0F0C5F008E60886F07F9E
:200A6E00011201D1F0A3C5F0F0C5F07F011201DFE98AF0C0E0C0F0740275F000C0E0C0F046
:200A8E0012051215811581158115817F001201D1F078FB120048E60886F0C0E0C0F074304F
:200AAE0075F000C0E0C0F07402C0E0C0F01238AC7FFA1200547F031201D112007589828A56
:200ACE0083E07003020B0F7F031201D11200757F001201D1E089828A8312006A2B7F001296
:200AEE0001D1F07F031201D1E0A3F5F0E0C5F012012B7F031201D1F0A3C5F0F0C5F0020A26
:200B0E00C37F001201D1E0F4047F001201D1F078FB12004886010886027F001201D1E075DA
:200B2E00F0007B047C00120119C001C002903C6512007512007C89828A83E0D083D082F03A
:200B4E0078FB120048E60886F02401C5F03400C5F0F9AAF07F001201D1E0540FC001C002D7
:200B6E00903C6512007512008C12007C89828A83E0D083D082F07F001201D1E012008C54C1
:200B8E00FFC5F05400C5F07F050201EB90A455E06003020C40748C75F0A3C0E0C0F0E4C002
:200BAE00E0C0E074C975F000C0E0C0F01238AC7FFA12005490A38BE075F0007B007C0012D4
:200BCE00018D7003020C2C798C7AA3742489828A83F0E4A20992E0F51F748C75F0A3C0E04D
:200BEE00C0F0E51F600774FC75F03C8005740075F03DC0E0C0F012390815811581158115A6
:200C0E0081748C75F0A3C0E0C0F0745675F0A4C0E0C0F01239081581158115811581748C1F
:200C2E0075F0A3C0E0C0F01239461581158190A455F078FB120048E60886F07B0A7C0012D4
:200C4E00016E700C18E60886F07BFF7C0012016E45F07003020CD1E4A20992E0F51F700399
:200C6E00020C94748C75F0A3C0E0C0F0748C75F0A32401C5F03400C0F0C0E0120A4C158108
:200C8E00158115811581748C75F0A3C0E0C0F01204541581158178FB120048E60886F07BEA
:200CAE000A7C0012016E7003020CC9740A75F000C0E0C0F01202E615811581E490A455F01F
:200CCE00020CFD748C75F0A390A45512006A2BC5F03400C5F0F9AAF078FB120048E6088651
:200CEE00F089828A83F090A455E00490A455F02278FB120048860108860289828A83E0709A
:200D0E0003020D3F18860108860289828A83E012008CC0E0C0F0120B9A1581158178FB12F7
:200D2E000048E60886F012012B18F608A6F0020CFE227FFA7EFF1201EDE4F5F07F0212018E
:200D4E00D1F0A3C5F0F0C5F078FB120048E60886F07F001201D1F0A3C5F0F0C5F0E47F04DF
:200D6E001201D1F07F041201D1E075F0007B027C0012017F7003020FC07F041201D1E0755A
:200D8E00F000900F96020095C2097F001201D1E0A3F5F0E0C5F012012B7F001201D1F0A32A
:200DAE00C5F0F0C5F0120139F9AAF089828A83E012008C900F0D0200957F001201D112009E
:200DCE007589828A83E012008C7B2012008312016E7003020DEF74017F041201D1F0020DFD
:200DEE00F774037F041201D1F0020F1978FB120048E60886F0C0E0C0F018E60886F02401D4
:200E0E00C5F03400C0F0C0E0120A4C15811581158115817F051201D1F07F051201D1E070BB
:200E2E0003020EAD74037F041201D1F0742F75F075C0E0C0F090A2BEE0A3F5F0E0C5F0124A
:200E4E00012B90A2BEF0A3C5F0F0C0F0C0E012398D158115811581158190A2BEF0A3C5F078
:200E6E00F0C5F090A38BE075F0007B027C0012016E7003020EAA740275F03DC0E0C0F07F2E
:200E8E00051201D1E075F000C0E0C0F0740275F0001237721581158115811581020EFF7F4A
:200EAE00001201D1E0A3F5F0E0C5F02402C5F03400C5F07F001201D1F0A3C5F0F0C5F07FB0
:200ECE00001201D112007589828A83E012008C7B2012008312016E7003020EF774017F04E0
:200EEE001201D1F0D209020EFF74037F041201D1F0020F1974037F041201D1F0020F19FA3C
:200F0E000D2300C70D21000000020F020FA2745675F0A4C0E0C0F07F001201D1E0A3F5F0EC
:200F2E00E0C0F0C0E0745675F0A4C0E0C0F012394615811581C0E0C0F01207627FFA12003D
:200F4E005445F07003020F6174037F041201D1F0020F9374027F041201D1F0745675F0A403
:200F6E00C0E0C0F0123946158115817F001201D112006E2BC5F03CC5F07F021201D1F0A3AA
:200F8E00C5F0F0C5F0020FA21C0F0100960D00000000A20F7F001201D1E0A3F5F0E0C5F056
:200FAE0012012B7F001201D1F0A3C5F0F0C5F0020D727F021201D1E0A3F5F0E0C5F07F062D
:200FCE000201EB7FFD7EFF1201EDE4F5F07F011201D1F0A3C5F0F0C5F012035745F07003EE
:200FEE000212741203CE7F001201D1F0E4A20892E0F51F700302101A7F001201D1E012001D
:20100E008CC0E0C0F01202E61581158190A2BDE0600302104274F475F0A1C0E0C0F0E4C0D8
:20102E00E0C0E074C975F000C0E0C0F01238AC7FFA1200547F001201D1E012008C9010BA20
:20104E0002009590A2BDE0700302107390A2BDE01490A2BDF079F47AA112008C12007CE4CA
:20106E0089828A83F00210C60210C674F475F0A190A2BD12006A2BC5F03400C5F0F9AAF075
:20108E007F001201D1E089828A83F090A2BDE00490A2BDF075F0007BC87C00120195700306
:2010AE000210B774C790A2BDF00210C676100A0051100800000079107F001201D1E0120090
:2010CE008C7B0A12008312016E700302127490A38BE075F00090125B02009579F47AA18938
:2010EE00828A83E012008C7B2A120083120176700302111374F475F0A17F011201D1F0A314
:20110E00C5F0F0C5F002126F74F475F0A1C0E0C0F0120D40158115817F011201D1F0A3C5DF
:20112E00F0F0C5F002126F90A2BDE070030211B279F47AA189828A83E012008C9011A2021F
:20114E0000950211B2741975F03DC0E0C0F01204541581158174F475F0A1C0E0C0F012043E
:20116E005415811581741B75F03DC0E0C0F01204541581158174F475F0A1C0E0C0F0120DED
:20118E0040158115817F011201D1F0A3C5F0F0C5F00211B250112D0050112A005011240021
:2011AE000000531102126F90A2BDE0700302124579F47AA189828A83E012008C90123502A8
:2011CE00009502124574F475F0A1C0E0C0F0120D40158115817F011201D1F0A3C5F0F0C569
:2011EE00F07F011201D1E0A3F5F0E0C5F045F07003021232741D75F03DC0E0C0F0120454B5
:20120E0015811581745675F0A4C0E0C0F012045415811581742175F03DC0E0C0F0120454EA
:20122E0015811581021245D0112D00D0112A00D01124000000D31102126F740175F000C0FC
:20124E00E0C0F01209F91581158102126FB51103003511020016110100E9100000000048B3
:20126E0012E490A2BDF07F011201D1E0A3F5F0E0C5F07F030201EB90A38BE075F0007B003C
:20128E007C0012016E700E90A38BE075F0007B027C0012016E45F070030212BE78FB120049
:2012AE0048E60886F0C0E0C0F0120CFE158115812290A38BE075F0007B007C0012016E70CF
:2012CE00030212F2745675F0A4C0E0C0F012045415811581742575F03DC0E0C0F012045449
:2012EE0015811581227FFD7EFF1201ED78FB120048E60886F02401C5F03400C5F0F9AAF012
:20130E0089828A83E012008C7B3D12008312016E700302144E18E60886F02402C5F03400F9
:20132E00C5F07F001201D1F0A3C5F0F0C5F07F001201D1E0A3F5F0E0C0F0C0E012394615F9
:20134E008115817B017C00120168700302143B745675F0A4C0E0C0F0E4C0E0C0E0741275EF
:20136E00F000C0E0C0F01238AC7FFA120054E47F021201D1F07F021201D1E075F0007B10DC
:20138E007C0012017F600D7F001201D112007589828A83E070120213F87F021201D1E0040A
:2013AE007F021201D1F080CD7F021201D1E079567AA412008C12007C7F001201D1E0A3F544
:2013CE00F0E0C5F012012B7F001201D1F0A3C5F0F0C5F0120139C001C002F9AAF089828AF5
:2013EE0083E0D083D082F00213A7745675F0A4C0E0C0F0745675F0A4C0E0C0F0123946153F
:20140E00811581D004D0032BC5F03CC5F0F9AAF0742089828A83F012175B746875F0A4C0D7
:20142E00E0C0F01208191581158102144B742775F03DC0E0C0F0121285158115810214993D
:20144E0012175B746875F0A4C0E0C0F01208191581158174C075F0A2C0E0C0F0744175F0C1
:20146E003DC0E0C0F0745675F0A4C0E0C0F0740375F0001237837FFA12005474C075F0A2EC
:20148E00C0E0C0F0120CFE158115817F030201EB78FB120048E60886F018F608A6F074C025
:2014AE0075F0A2C0E0C0F0745475F03DC0E0C0F0745675F0A4C0E0C0F0740375F0001237C5
:2014CE00837FFA12005474C075F0A2C0E0C0F0120CFE15811581788018E660FC881F74C09C
:2014EE0075F0A2C0E0C0F0746575F03DC0E0C0F0E51F75F000C0E0C0F0747FC0E0C0F0744C
:20150E000475F0001237837FF812005474C075F0A2C0E0C0F0120CFE158115812278FB1231
:20152E000048E60886F018F608A6F074C075F0A2C0E0C0F0747F75F03DC0E0C0F0E50A7571
:20154E00F000C0E0C0F090A2BEE0A3F5F0E0C0F0C0E0740475F0001237837FF812005474BB
:20156E00C075F0A2C0E0C0F0120CFE15811581E4F50AE4F5F090A2BEF0A3C5F0F0C5F02253
:20158E007FFE7EFF1201ED78FB120048E60886F02401C5F03400C5F07F001201D1F0A3C594
:2015AE00F0F0C5F07F001201D112007589828A83E012008CC0E0C0F0123866158115814597
:2015CE00F070030215F07F001201D1E0A3F5F0E0C0F0C0E01238CF1581158190A667F002C4
:2015EE00162A74C075F0A2C0E0C0F074AE75F03DC0E0C0F090A667E075F000C0E0C0F07458
:20160E000375F0001237837FFA12005474C075F0A2C0E0C0F0120CFE158115817F02020152
:20162E00EB7FFE7EFF1201ED78FB120048E60886F02401C5F03400C5F07F001201D1F0A3CD
:20164E00C5F0F0C5F07F001201D112007589828A83E012008C9016FE02009574C075F0A22C
:20166E00C0E0C0F074C275F03DC0E0C0F090A38BE075F000C0E0C0F0740375F000123783E9
:20168E007FFA12005474C075F0A2C0E0C0F0120CFE158115810217067F001201D112007581
:2016AE0089828A83E012008CC0E0C0F01238661581158145F070030216EB7F001201D1E06C
:2016CE00A3F5F0E0C0F0C0E01238CF15811581C0E0C0F01209F9158115810216FB74D275A1
:2016EE00F03DC0E0C0F012128515811581021706691600000000A6167F020201EB90A38B03
:20170E00E075F0007B007C0012016E700302175A74C075F0A2C0E0C0F074EA75F03DC0E0ED
:20172E00C0F078F7120048E60886F0C0E0C0F0740375F0001237837FFA12005474C075F04E
:20174E00A2C0E0C0F012128515811581227FFF7EFF1201ED745675F0A4C0E0C0F0123946E3
:20176E00158115817F001201D1F07F001201D1E075F0007B027C0012017F70030217C674E3
:20178E005675F0A4C0E0C0F0745F75F03CC0E0C0F0741175F000C0E0C0F0123A0C7FFA12AB
:2017AE000054745675F0A4C0E0C0F0123946158115817F001201D1F07F001201D1E0C394FA
:2017CE000279567AA412008C12007C89828A83E0F51FD2B3A2B3B392E0F51F7F001201D15E
:2017EE00E0C3940279567AA412008C12007CE51F89828A83F07F010201EBD2B2E4A2B292C1
:20180E00E0F51F7003021829740175F000C0E0C0F01209F915811581021835E4C0E0C0E033
:20182E001209F915811581227FF87EFF1201ED749E75F0A5C0E0C0F074F475F0A1C0E0C00A
:20184E00F0123918158115811581158178FB120048E60886F07F021201D1F0A3C5F0F0C53C
:20186E00F07F001201D1F0A3C5F0F0C5F07F001201D112007589828A83E0700302192D7FFE
:20188E00001201D112007589828A83E012008C7B2012008312016E70030218C87F001201A1
:2018AE00D1E0A3F5F0E0C5F012012B7F001201D1F0A3C5F0F0C5F002192A7F021201D11202
:2018CE000075C001C0027F001201D112007589828A83E012008CC0E0C0F012387A158115C3
:2018EE0081D083D082F07F001201D1E0A3F5F0E0C5F012012B7F001201D1F0A3C5F0F0C5C6
:20190E00F07F021201D1E0A3F5F0E0C5F012012B7F021201D1F0A3C5F0F0C5F002187B7FC3
:20192E00021201D1120075E489828A83F078FB120048E60886F02401C5F03400C5F07F00CD
:20194E001201D1F0A3C5F0F0C5F018860108860289828A83E012008C901D7D02009578FBAF
:20196E00120048E60886F0C0E0C0F01212F315811581021DAD12149E74C075F0A2C0E0C0DD
:20198E00F0740575F03EC0E0C0F0E51675F000C0E0C0F074031237837FFA12005474C07562
:2019AE00F0A2C0E0C0F0120CFE15811581021DAD78FB120048E60886F0C0E0C0F012152B50
:2019CE0015811581021DAD78FB120048E60886F0C0E0C0F012158E15811581021DAD78FB60
:2019EE00120048E60886F0C0E0C0F012162F15811581021DAD7F001201DFE98AF0C0E0C048
:201A0E00F07F041201DFE98AF0C0E0C0F07F061201DFE98AF0C0E0C0F0122D777FFA120035
:201A2E005445F06003021A5D7F041201D1E0A3F5F0E0C0F0C0E07F061201D1E0A3F5F0E083
:201A4E00C0F0C0E012303C1581158115811581740A75F000C0E0C0F0120B9A15811581023A
:201A6E001DAD7F001201D1E0A3F5F0E0C0F0C0E0741175F03EC0E0C0F0123A57158115814C
:201A8E001581158145F07003021B1B7F001201D112007589828A83E012008CC0E0C0F0124A
:201AAE0038661581158145F07003021ADD7F001201D1E0A3F5F0E0C0F0C0E01238CF158103
:201ACE00158190A47EF0A3C5F0F0C5F0021B1874C075F0A2C0E0C0F0741675F03EC0E0C076
:201AEE00F090A47EE0A3F5F0E0C0F0C0E0740375F0001237837FFA12005474C075F0A2C01C
:201B0E00E0C0F0120CFE15811581021B21120399020000021DAD7F001201D1120075898230
:201B2E008A83E07003021B9B7F001201DFE98AF0C0E0C0F07F041201DFE98AF0C0E0C0F033
:201B4E00122949158115811581158145F06003021B9B7F001201D112007589828A83E01257
:201B6E00008C7B2C12008312016E7003021B987F001201D1E0A3F5F0E0C5F012012B7F00C9
:201B8E001201D1F0A3C5F0F0C5F0021B24021DAD7F001201DFE98AF0C0E0C0F01224B11539
:201BAE008115817F041201D1F0A3C5F0F0C5F07F041201D1E0A3F5F0E0C5F07B007C8012BF
:201BCE0001767003021C8D749E75F0A5C0E0C0F0743D75F000C0E0C0F0123A8D158115818B
:201BEE00158115817F001201D1F0A3C5F0F0C5F07F001201D1E0A3F5F0E0C5F045F0603630
:201C0E007F001201D112007589828A83E012008C7B3D12008312016E601C7F001201D1E0A9
:201C2E00A3F5F0E0C0F0C0E0123946158115817B017C0012016045F07003021C7D7F0012E2
:201C4E0001D1E0A3F5F0E0C5F02401C5F03400C0F0C0E07F041201D1E0A3F5F0E0C0F0C02A
:201C6E00E01232D91581158115811581021C8D743175F03EC0E0C0F01212851581158102E7
:201C8E001DAD021DAD745275F03EC0E0C0F0120CFE15811581748775F03EC0E0C0F0120C93
:201CAE00FE1581158174B475F03EC0E0C0F0120CFE1581158174F375F03EC0E0C0F0120C11
:201CCE00FE15811581741D75F03FC0E0C0F0120CFE15811581744B75F03FC0E0C0F0120C2E
:201CEE00FE15811581746B75F03FC0E0C0F0120CFE15811581748775F03FC0E0C0F0120C84
:201D0E00FE1581158174BC75F03FC0E0C0F0120CFE1581158174ED75F03FC0E0C0F0120CAC
:201D2E00FE15811581740775F040C0E0C0F0120CFE15811581742D75F040C0E0C0F0120CFF
:201D4E00FE15811581744C75F040C0E0C0F0120CFE15811581021DAD78FB120048E6088641
:201D6E00F0C0E0C0F012170B15811581021DAD931C3F00901C00009E1B5400241B53007040
:201D8E001A5200031A5100EC194E00D5194C00BE194500831944006C1941000000661D7F0A
:201DAE00080201EBE4F522E4F516740E75F0DCF51485F015E58854CFF588E58954F0F589A2
:201DCE004401F589E4F58AF58CD2A9D28C22C0E0C0D0C28C85148A85158CD28C05170516F7
:201DEE00E516B464004006D217249CF516D0D0D0E032227FFF7EFF1201EDE5167F0012019C
:201E0E00D1F07F001201D1E075F000AB167C0012016E6003021E1078FB120048E60886F0C9
:201E2E0012013918F608A6F012012B45F06003021E087F010201EB78FB120048E60886F0FF
:201E4E0045F07003021E7375F02ED5F0FD78FB120048E60886F012013918F608A6F045F086
:201E6E006003021E552290A667E054207003021EEB74C075F0A2C0E0C0F0746875F040C01F
:201E8E00E0C0F078F7120048E60886F0C0E0C0F078F1120048E60886F0C333C5F033C5F06D
:201EAE00795B7A3C12007C89828A83E0A3F5F0E0C5F078F312004826C5F00836C0F0C0E0B9
:201ECE00740475F0001237837FF812005474C075F0A2C0E0C0F01212851581158178F7128D
:201EEE000048E60886F0C333C5F033C5F02400C5F03400C5F079807AA412007C89828A8316
:201F0E00E0A3F5F0E0C5F05408C5F05400C5F045F0700302202D78F7120048E60886F0C3B5
:201F2E0033C5F033C5F0795B7A3C12007C89828A83E0A3F5F0E0C5F090201E02009578F7C2
:201F4E00120048E60886F00826C5F00836C5F079827AA412007C89828A83E075F00078FB68
:201F6E0012004856C5F00856C5F089828A83F078F7120048E60886F00826C5F00836C5F0D0
:201F8E0079827AA412007C78FB120048E60886F089828A8312006A4B18F608A6F018E608CA
:201FAE0086F0F59002202A78F7120048E60886F00826C5F00836C5F079827AA412007C8999
:201FCE00828A83E075F00078FB12004856C5F00856C5F089828A83F078F7120048E60886EF
:201FEE00F00826C5F00836C5F079827AA412007C78FB120048E60886F089828A8312006AA1
:20200E004B18F608A6F018E60886F0F5B002202AB51F03004C1F010000002A2002207178B6
:20202E00F7120048E60886F0C333C5F033C5F0795B7A3C12007C89828A83E0A3F5F0E0C50D
:20204E00F078F912004826C5F00836C0F0C0E008E60886F0C0E0C0F0123ACB15811581153A
:20206E00811581C2B5740275F000C0E0C0F0121E4515811581D2B578F7120048E60886F044
:20208E00C333C5F033C0F0C0E008E60886F0C333C5F033C5F0D004D0032BC5F03CC5F07914
:2020AE00807AA412007C89828A83E0A3F5F0E0C5F05410C5F05400C5F045F07003022111D3
:2020CE0078F7120048E60886F0C333C5F033C0F0C0E008E60886F0C333C5F033C5F0D004C4
:2020EE00D0032BC5F03CC5F079837AA412007C78FB120048E60886F089828A83F0A3C5F0F5
:20210E00F0C5F0227FFD7EFF1201ED78F9120048E60886F0C333C5F033C0F0C0E008E6089E
:20212E0086F0C333C5F033C5F0D004D0032BC5F03CC5F079807AA412007C89828A83E0A3D0
:20214E00F5F0E0C5F05410C5F05400C5F045F070030221B378F9120048E60886F0C333C56D
:20216E00F033C0F0C0E008E60886F0C333C5F033C5F0D004D0032BC5F03CC5F079837AA44D
:20218E0012007C89828A83E0A3F5F0E0C5F07F001201D1F0A3C5F0F0C5F074017F02120135
:2021AE00D1F0022295E47F021201D1F078F9120048E60886F0C333C5F033C5F02400C5F0C3
:2021CE003400C5F079807AA412007C89828A83E0A3F5F0E0C5F05408C5F05400C5F045F0FF
:2021EE00700302225278F9120048E60886F0C333C5F033C5F0795B7A3C12007C89828A83F6
:20220E00E0A3F5F0E0C5F0902243020095E59075F0007F001201D1F0A3C5F0F0C5F00222D9
:20222E004FE5B075F0007F001201D1F0A3C5F0F0C5F002224F2F2203001B22010000004FA3
:20224E002202229578F9120048E60886F0C333C5F033C5F0795B7A3C12007C89828A83E0C3
:20226E00A3F5F0E0C5F078FB12004826C5F00836C0F0C0E0123AAA158115817F001201D178
:20228E00F0A3C5F0F0C5F090A667E05420700302232574C075F0A2C0E0C0F0748475F0406D
:2022AE00C0E0C0F07F001201D1E0A3F5F0E0C0F0C0E078F3120048E60886F0C333C5F033BE
:2022CE00C5F0795B7A3C12007C89828A83E0A3F5F0E0C5F078F512004826C5F00836C0F07E
:2022EE00C0E07F021201D1E0600774A475F040800574AA75F040C0E0C0F0740575F000123F
:20230E0037837FF612005474C075F0A2C0E0C0F0120CFE158115817F001201D1E0A3F5F07C
:20232E00E0C5F07F030201EB7FFF7EFF1201ED741090A47DF074AB75F040C0E0C0F0121232
:20234E008515811581748075F0A4C0E0C0F0E4C0E0C0E0740275F000C0E0C0F01238AC7FAD
:20236E00FA120054748275F0A4C0E0C0F074FF75F000C0E0C0F07401C0E0C0F01238AC7F3E
:20238E00FA120054745E75F00190A47EF0A3C5F0F0C5F0E47F001201D1F07F001201D1E07E
:2023AE0075F0007B017C0012017F70120224AC7F001201D1E0047F001201D1F080DC74C0A2
:2023CE0075F0A2C0E0C0F074CC75F040C0E0C0F07F001201D1E075F000C333C5F033C5F028
:2023EE0079597A3C12007C89828A83E0A3F5F0E0C0F0C0E0740375F0001237837FFA1200D6
:20240E005474C075F0A2C0E0C0F0121285158115817F001201D1E075F000C333C5F033C5AF
:20242E00F02400C5F03400C5F079807AA412007C89828A83E0A3F5F0E0C5F04401C5F044E4
:20244E0000C5F089828A83F0A3C5F0F0C5F07F001201D1E075F000C333C5F033C5F0240055
:20246E00C5F03400C5F079807AA412007C89828A83E0A3F5F0E0C5F04408C5F04400C5F0FC
:20248E0089828A83F0A3C5F0F0C5F074D575F040C0E0C0F0121285158115810223BD7F01B4
:2024AE000201EB7FF87EFF1201EDE47F061201D1F07F051201D1F0E475F0E07F001201D10B
:2024CE00F0A3C5F0F0C5F0748575F0A4C0E0C0F0E4C0E0C0E074C975F000C0E0C0F012384F
:2024EE00AC7FFA120054748575F0A47F021201D1F0A3C5F0F0C5F078FB120048860108860D
:20250E000289828A8312007589828A83E012008CC0E0C0F01238321581158145F06024784D
:20252E00FB120048860108860289828A8312007589828A83E012008CC0E0C0F012385015ED
:20254E0081158145F070030225CC7F021201D1E0A3F5F0E0C5F012012B7F021201D1F0A323
:20256E00C5F0F0C5F0120139F9AAF0C001C00278F9120048860108860289828A8312007510
:20258E0089828A83E012008CC0E0C0F012387A15811581D083D082F078FB12004886010866
:2025AE00860289828A83E0A3F5F0E0C5F012012B89828A83F0A3C5F0F0C5F0022505E47F9E
:2025CE00041201D1F07F041201D1E075F0007B017C0012017F70120226397F041201D1E0B5
:2025EE00047F041201D1F080DC748575F0A4C0E0C0F07F041201D1E075F000C333C5F0333A
:20260E00C5F079597A3C12007C89828A83E0A3F5F0E0C0F0C0E0123A5715811581158115B7
:20262E008145F070030226390225E87F041201D1E075F0007B017C0012016E7003022689AA
:20264E0074C075F0A2C0E0C0F074DD75F040C0E0C0F0748575F0A4C0E0C0F0740375F0006D
:20266E001237837FFA12005474C075F0A2C0E0C0F0121285158115810228E77F001201D1CD
:20268E00E0A3F5F0E0C5F054FFC5F0547FC5F07F001201D1F0A3C5F0F0C5F090A667E0547E
:2026AE002070030226EC74C075F0A2C0E0C0F074F775F040C0E0C0F0748575F0A4C0E0C018
:2026CE00F0740375F0001237837FFA12005474C075F0A2C0E0C0F0120CFE15811581E47F3F
:2026EE00051201D1F07F001201D1E0A3F5F0E0C5F054FFC5F054BFC5F07F001201D1F0A3CD
:20270E00C5F0F0C5F078FB120048860108860289828A8312007589828A83E012008C7B2E8F
:20272E0012008312016E70030228CC18860108860289828A83E0A3F5F0E0C5F012012B8901
:20274E00828A83F0A3C5F0F0C5F018E60886F0C0E0C0F012062F158115817F071201D1F056
:20276E007F071201D1E075F0007B107C0012017F60327F041201D1E075F000C333C5F033E7
:20278E00C5F02400C5F03400C5F079807AA412007C89828A83E0A3F5F0E0C5F05402C5F0EF
:2027AE005400C5F045F070477F071201D1E075F0007B087C0012017F60357F041201D1E0FA
:2027CE0075F000C333C5F033C5F02400C5F03400C5F079807AA412007C89828A83E0A3F5FC
:2027EE00F0E0C5F05402C5F05400C5F012014C45F0700302287A7F001201D1E0A3F5F0E0DC
:20280E00C5F054FFC5F054DFC5F07F001201D1F0A3C5F0F0C5F07F071201D1E07F061201D3
:20282E00D1F090A667E05420700302287774C075F0A2C0E0C0F0740275F041C0E0C0F07F4E
:20284E00071201D1E075F000C0E0C0F0740375F0001237837FFA12005474C075F0A2C0E088
:20286E00C0F0120CFE158115810228C9E475F0807F001201D1F0A3C5F0F0C5F074C075F0AD
:20288E00A2C0E0C0F0741275F041C0E0C0F07F071201D1E075F000C0E0C0F0740375F000E1
:2028AE001237837FFA12005474C075F0A2C0E0C0F0121285158115810228E70228E790A6A7
:2028CE0067E0542070030228E7742775F041C0E0C0F0120CFE158115817F041201D1E07516
:2028EE00F0007B087C0012010BC0E0C0F07F051201D1E075F0007B047C0012010BD004D003
:20290E00034BC5F04CC5F07F061201D112006A4B7F001201D112006E4BC5F04CC5F07F0012
:20292E001201D1F0A3C5F0F0C5F07F001201D1E0A3F5F0E0C5F07F080201EB7FF57EFF12E0
:20294E0001ED740175F0007F001201D1F0A3C5F0F0C5F078FB1200488601088602C001C0EC
:20296E0002181818E60886F0C0E0C0F01224B1158115817F021201D1F0A3C5F0F0C5F0D016
:20298E0083D082F0A3C5F0F0C5F07F021201D1E0A3F5F0E0C5F05400C5F05480C5F045F03E
:2029AE006003022D667F021201D1E0A3F5F0E0C5F05400C5F0540FC5F07B087C0012011963
:2029CE007F041201D1F07F021201D1E0A3F5F0E0C5F054F0C5F05400C5F07B047C00120120
:2029EE00197F051201D1F07F021201D1E0A3F5F0E0C5F0540FC5F05400C5F07F061201D16C
:202A0E00F078F9120048860108860289828A8312007589828A83E012008C7B3D1200831242
:202A2E000176702718860108860289828A83E0A3F5F0E0C5F02401C5F03400C5F0F9AAF0E0
:202A4E0089828A83E012008C12014C45F07003022A73742A75F041C0E0C0F0121285158159
:202A6E001581022D6678F9120048860108860289828A83E0A3F5F0E0C5F012012B89828A53
:202A8E0083F0A3C5F0F0C5F07F021201D1E0A3F5F0E0C5F05400C5F05440C5F045F070035C
:202AAE00022AC4744875F041C0E0C0F012128515811581022D6690A47DE075F000902B2427
:202ACE0002009578F9120048E60886F0C0E0C0F0740475F000C0E0C0F01205121581158150
:202AEE00158115817F071201D1F0A3C5F0F0C5F0022B3078F9120048E60886F0C0E0C0F069
:202B0E0012062F158115817F071201D1F0A3C5F0F0C5F0022B30012B0A00D12A100000003F
:202B2E00D12A7F021201D1E0A3F5F0E0C5F05400C5F05420C5F045F07003022B7E7F041210
:202B4E0001D1E075F000C0E0C0F07F051201D1E075F000C0E0C0F07F071201D1E0A3F5F031
:202B6E00E0C0F0C0E0121E747FFA120054022D577F071201D1E0A3F5F0E0C5F07B017C00AF
:202B8E0012018D7003022BA9745D75F041C0E0C0F012128515811581022D667F041201D1A6
:202BAE00E075F000C333C5F033C5F02400C5F03400C5F079807AA412007C89828A83E0A32D
:202BCE00F5F0E0C5F05408C5F05400C5F045F07003022C5A7F041201D1E07F051201D11262
:202BEE00006A2B79827AA475F00012007C740175F0007F061201D112006A7C0012010BF4D9
:202C0E0089828A8312006A5B89828A83F07F041201D1E07F051201D112006A2B79827AA440
:202C2E0075F00012007C7F071201D1E0A3F5F0E0C5F07F061201D112006A7C0012010B8924
:202C4E00828A8312006A4B89828A83F07F041201D1E075F000C0E0C0F07F051201D1E0754F
:202C6E00F000C0E0C0F012211215811581158115817F091201D1F0A3C5F0F0C5F074017526
:202C8E00F0007F061201D112006A7C0012010BF475F0007F091201D112006E5BC5F05CC541
:202CAE00F07F091201D1F0A3C5F0F0C5F07F071201D1E0A3F5F0E0C5F07F061201D11200DB
:202CCE006A7C0012010B7F091201D112006E4BC5F04CC5F07F091201D1F0A3C5F0F0C5F09C
:202CEE007F041201D1E07F051201D112006A2B79827AA475F00012007C7F091201D1E0A375
:202D0E00F5F0E0C5F089828A8312006A4B7F091201D1F0A3C5F0F0C5F07F041201D1E07537
:202D2E00F000C0E0C0F07F051201D1E075F000C0E0C0F07F091201D1E0A3F5F0E0C0F0C024
:202D4E00E0121E747FFA120054E4F5F07F001201D1F0A3C5F0F0C5F07F001201D1E0A3F50E
:202D6E00F0E0C5F07F0B0201EB7FF77EFF1201ED78F91200488601088602C001C0021818C0
:202D8E0018E60886F0C0E0C0F01224B1158115817F021201D1F0A3C5F0F0C5F0D083D0824F
:202DAE00F0A3C5F0F0C5F0740175F0007F001201D1F0A3C5F0F0C5F0E4F5F07F071201D1BB
:202DCE00F0A3C5F0F0C5F07F021201D1E0A3F5F0E0C5F05400C5F05480C5F045F06003026A
:202DEE00300A7F021201D1E0A3F5F0E0C5F05400C5F0540FC5F07B087C001201197F041248
:202E0E0001D1F07F021201D1E0A3F5F0E0C5F054F0C5F05400C5F07B047C001201197F05D3
:202E2E001201D1F07F021201D1E0A3F5F0E0C5F0540FC5F05400C5F07F061201D1F07F0451
:202E4E001201D1E075F000C333C5F033C5F02400C5F03400C5F079807AA412007C89828AAC
:202E6E0083E0A3F5F0E0C5F05401C5F05400C5F045F06003022EDB74C075F0A2C0E0C0F083
:202E8E00747B75F041C0E0C0F07F041201D1E075F000C333C5F033C5F079597A3C12007CEA
:202EAE0089828A83E0A3F5F0E0C0F0C0E0740375F0001237837FFA12005474C075F0A2C0D2
:202ECE00E0C0F01212851581158102300A78F7120048860108860289828A831200758982B9
:202EEE008A83E012008C7B3D12008312016E7003022F14749875F041C0E0C0F012128515F3
:202F0E0081158102300A7F021201D1E0A3F5F0E0C5F05400C5F05440C5F045F07003022FC3
:202F2E0036E47F051201D1F07F021201D1E0A3F5F0E0C5F05400C5F05420C5F045F07003D5
:202F4E00022F857F041201D1E075F000C0E0C0F07F051201D1E075F000C0E0C0F01221126F
:202F6E0015811581158115817F071201D1F0A3C5F0F0C5F0022FFB7F041201D1E075F000BC
:202F8E00C0E0C0F07F051201D1E075F000C0E0C0F012211215811581158115817F071201A0
:202FAE00D1F0A3C5F0F0C5F07F071201D1E0A3F5F0E0C5F07F061201D112006A7C0012016A
:202FCE00197F071201D1F0A3C5F0F0C5F07F071201D1E0A3F5F0E0C5F05401C5F05400C5E9
:202FEE00F07F071201D1F0A3C5F0F0C5F0E4F5F07F001201D1F0A3C5F0F0C5F078FB1200DE
:20300E004886010886027F071201D1E0A3F5F0E0C5F089828A83F0A3C5F0F0C5F07F001246
:20302E0001D1E0A3F5F0E0C5F07F090201EB7FF97EFF1201ED740175F0007F001201D1F01B
:20304E00A3C5F0F0C5F078F9120048E60886F05400C5F05480C5F045F0700302308C74C00A
:20306E0075F0A2C0E0C0F074AE75F041C0E0C0F0123918158115811581158102329278F9E1
:20308E00120048E60886F05400C5F0540FC5F07B087C001201197F021201D1F018E6088637
:2030AE00F054F0C5F05400C5F07B047C001201197F031201D1F018E60886F0540FC5F054AB
:2030CE0000C5F07F041201D1F074C075F0A2C0E0C0F07F021201D1E075F000C333C5F033C3
:2030EE00C5F079597A3C12007C89828A83E0A3F5F0E0C0F0C0E0123918158115811581150D
:20310E008178F9120048E60886F05400C5F05420C5F045F0600302316F74C075F0A2C0E0AA
:20312E00C0F074C075F0A2C0E0C0F012394615811581D004D0032BC5F03CC0F0C0E074BE44
:20314E0075F041C0E0C0F07F041201D1E075F000C0E0C0F0740375F0001237837FFA12003C
:20316E005474C075F0A2C0E0C0F074C275F041C0E0C0F0123908158115811581158178F91A
:20318E00120048E60886F05400C5F05420C5F045F060030231B874C475F0417F051201D168
:2031AE00F0A3C5F0F0C5F002323690A47DE075F00090322A0200957F021201D1E075F00087
:2031CE00C333C5F033C5F02400C5F03400C5F079807AA412007C89828A83E0A3F5F0E0C5C2
:2031EE00F05402C5F05400C5F045F0600774C775F041800574CC75F0417F051201D1F0A3DA
:20320E00C5F0F0C5F002323674D175F0417F051201D1F0A3C5F0F0C5F002323616320A00E0
:20322E00C53110000000C53174C075F0A2C0E0C0F074C075F0A2C0E0C0F012394615811532
:20324E0081D004D0032BC5F03CC0F0C0E07F051201D1E0A3F5F0E0C0F0C0E078F712004803
:20326E00E60886F0C0E0C0F0740375F0001237837FFA120054E4F5F07F001201D1F0A3C581
:20328E00F0F0C5F07F001201D1E0A3F5F0E0C5F045F070030232B874C075F0A2C0E0C0F00C
:2032AE00121285158115810232C874C075F0A2C0E0C0F0120CFE158115817F001201D1E019
:2032CE00A3F5F0E0C5F07F070201EB7FF07EFF1201ED78F9120048860108860289828A8369
:2032EE00E070030236A218860108860289828A83E012008C7B5C12008312016E7003023636
:20330E001A18E60886F02401C5F03400C5F0F9AAF089828A83E012008CC0E0C0F0123893F0
:20332E0015811581903529020095E4F5F07F021201DF12007C78F9120048E60886F02402AF
:20334E00C5F03400C5F0C001C002F9AAF089828A83E0541FD083D082F0740175F0007F0250
:20336E001201DF12007CE489828A83F078F9120048E60886F02401C5F03400C5F018F608CB
:20338E00A6F00235497F021201DFE98AF0C0E0C0F074D475F041C0E0C0F012391815811597
:2033AE0081158115810235497F021201DFE98AF0C0E0C0F074D675F041C0E0C0F012391809
:2033CE0015811581158115810235497F021201DFE98AF0C0E0C0F074D875F041C0E0C0F09F
:2033EE0012391815811581158115810235497F021201DFE98AF0C0E0C0F074DA75F041C0AA
:20340E00E0C0F0123918158115811581158102354978F9120048E60886F07F0C1201D1F045
:20342E00A3C5F0F0C5F018E60886F02402C5F03400C5F018F608A6F018E60886F07F0E127A
:20344E0001D1F0A3C5F0F0C5F0E4F5F07F021201DF12007CC001C0027F0E1201DFE98AF070
:20346E00C0E0C0F0740275F000C0E0C0F01205121581158115811581D083D082F0740175C3
:20348E00F0007F021201DF12007CE489828A83F07F0C1201D1E0A3F5F0E0C5F02402C5F0FA
:2034AE003400C5F078F9120048F608A6F0023549E4F5F07F021201DF12007C745C89828A07
:2034CE0083F0740175F0007F021201DF12007CE489828A83F0023549E4F5F07F021201DFE8
:2034EE0012007C78F9120048E60886F02401C5F03400C5F0C001C002F9AAF089828A83E030
:20350E00D083D082F0740175F0007F021201DF12007CE489828A83F0023549BE345C001F54
:20352E00347800FC337200D9336E00B633660093336500383363000000E63478F912004889
:20354E00E60886F02402C5F03400C5F018F608A6F07F021201DFE98AF07F0C1201D1F0A3B1
:20356E00C5F0F0C5F07F0C1201D112007589828A83E0700302361778FB120048E60886F002
:20358E005400C5F0540FC5F07B087C00120119C0E0C0F018E60886F054F0C5F05400C5F003
:2035AE007B047C00120119C0E0C0F07F0C1201D112007589828A83E012008CC0E0C0F01298
:2035CE001E747FFA1200547F0C1201D1E0A3F5F0E0C5F012012B7F0C1201D1F0A3C5F0F01B
:2035EE00C5F090A47EE0A3F5F0E0C5F045F0700302361490A47EE0A3F5F0E0C0F0C0E01209
:20360E001E451581158102357302369F78FB120048E60886F05400C5F0540FC5F07B087C3B
:20362E0000120119C0E0C0F018E60886F054F0C5F05400C5F07B047C00120119C0E0C0F00B
:20364E00181818860108860289828A83E012008CC0E0C0F0121E747FFA12005478F9120011
:20366E0048E60886F012012B18F608A6F090A47EE0A3F5F0E0C5F045F0700302369F90A444
:20368E007EE0A3F5F0E0C0F0C0E0121E45158115810232E07F001201D1E0A3F5F0E0C5F0F1
:2036AE007F100201EB7FFE7EFF1201ED1201F8121DB2120205D2AF12089390A38BE0600351
:2036CE0002370174DC75F041C0E0C0F0120CFE15811581740675F042C0E0C0F0120CFE1572
:2036EE00811581740B75F042C0E0C0F0120CFE158115811223361212BF740175F00045F08A
:20370E00700302375DE4A21792E0F51F7003023727C217B2B2B2B2B2B2120FD17F00120113
:20372E00D1F0A3C5F0F0C5F07B007C00120176700302375A7F001201D1E0A3F5F0E0C0F0DC
:20374E00C0E0121836158115811212BF023707743375F042C0E0C0F0120CFE158115817FA7
:20376E00020201EB23F42581F81201B9123AEB1201B902045E23F42581F88682088683088D
:20378E00023AEB000000000000000000202020202000000000000000000000000000000054
:2037AE00000000600101010101010101010101010101011818181818181818181801010199
:2037CE00010101010A0A0A0A0A0A0202020202020202020202020202020202020202010171
:2037EE00010101010C0C0C0C0C0C040404040404040404040404040404040404040401011D
:20380E00010100C2D578FB120048E6903791C2E79355F060027401A2D575F00092F065F0EB
:20382E0075F0002278FB120048E6A2E7B3E4F5F092E02275F00280CB75F00480C675F006DB
:20384E0080C175F01680BC75F01780B775F05780B2D2D575F05780AD75F01080A675F00829
:20386E0080A175F001809C75F020809778FB120048E6C0E008E6C0E012384613D0F0D0E007
:20388E00500224E02278FB120048E6C0E008E6C0E012384113D0F0D0E050E924202278F7A5
:2038AE00120048868208868308860708088603088604EB4C600AEFF0A31BBBFFF51C80F24C
:2038CE002278FB1200488682088683E4FBFCFFE0A3B42D030FE0A3C39430B40A005012FA5E
:2038EE00740A75F0001200BE2AFBE5F03400FC80E4EB8CF0DF030201432278F91200488677
:20390E0082088683E0600DA380FA78F91200488682088683088601088602C9C582C9CAC531
:20392E0083CAE0A3C9C582C9CAC583CAF06003A380E8E5828583F02278FB12004886820838
:20394E008683E4F5F0FAE06009A30ABA00F805F080F4EA2278FB120048E60886F030F73ADE
:20396E0002014378F91200488603088604088605088606ED8EF012019B401CED8EF022786C
:20398E00F91200488603088604088605088606ED8EF012019B40E4EB8CF02278FB120048F1
:2039AE00860308860485FEF0E5017F0012017F600575F001E422EF0FF5F0A412017F70F624
:2039CE00EF1475F00022123A2E123A3A123A41123A48E0F7A30980F7123A2E123A41123AE1
:2039EE003A123A48E7F009A380F7123A2E123A3A123A41A882123A48E6F7080980F7123AF5
:203A0E002E123A3A123A41123A48E0A3CAC583CAC9C582C9F0A3CAC583CAC9C582C980E7DC
:203A2E0078FA120048860418860318228683188682182286021886011822EB4C60061BBB10
:203A4E00FF011C22158115812278F91200488682088683088601088602C9C582C9CAC583DE
:203A6E00CAE0F5F0A3C9C582C9CAC583CAE0B5F0056009A380E37401500274FF02008C7818
:203A8E00F912004886820886830886F0E0B5F0068583F0E58222A370F3F5F02278FB120090
:203AAE00488682088683E075F0002278FB1200488682088683E0F5F0A3E0C5F02278F912A8
:203ACE000048868208868308E6F02278F9120048868208868308E608F0A3E6F022123C3292
:203AEE00868208868308E4FEFFE07006123C32E4F022B42551A3E0B42D05430780A3E0B456
:203B0E00300343074024D0B40A00500BCE75F00AA42EFEA3E080EEE0B46413E60886F03030
:203B2E00F708430720120143A6F018F68003B4750543070A8021B478054307108019B46F27
:203B4E00104307088011123C32F0A3123C32A38095B462624307027A00C004C005C006C0CC
:203B6E0007AB0753031F7C00E60886F01200D8A6F018F6EDD007D006D005D0042430B43A16
:203B8E000040022407C0E00AE645F070CC123C32A902EF30E505742DF0A30A123C3BD0E0FE
:203BAE00F0A3D9FA0808EF30E7A1EAC39E509C7420F0A30A80F4B4630DAA01123C32123C61
:203BCE003BE6F0A380DEB47331C082C08386820886837A00E06004A30A80F98683188682C2
:203BEE00123C32123C3B123C32E0A3123C326004F0A380F2D005D00480AAB4691B86017AB6
:203C0E0000E76004090A80F9123C32123C3B8601E76091F009A380F8F97A01123C32123C01
:203C2E003BE9809ECDC583CDCCC582CC22EE601A8FF020F715C002EAC39E500C742030F61B
:203C4E00027430F0A30A80EFD00222673C0100010044494F302000EB3C445000436F6E7391
:203C6E006F6C652073746174757320666C61677320253032780A00205472616E733A20203A
:203C8E004865616420253032782C205461696C20253032782C2043747220253032782C20B0
:203CAE004D617820253032780A00205265633A202020204865616420253032782C20546121
:203CCE00696C20253032782C2043747220253032782C204D617820253032780A0030313220
:203CEE0033343536373839414243444546003030200020002A2A2A204261642063686563AF
:203D0E006B73756D3A202532780A002A000A002A2120004F4B0A003E002A2A2A204E6F20A6
:203D2E006164647265737320737472696E672E2E2E0A004E6574206164647265737320698E
:203D4E00732025730A004E65742061646472657373205B25735D002E2020537461636B20FF
:203D6E007573656420253032782F253032782E0A004572726F7220666C6167732025303221
:203D8E00782E20204E6574776F726B20636865636B73756D206572726F72732025750A0051
:203DAE004C6F6767696E67206D6F64652069732025750A004E6574206D6F646520697320A1
:203DCE0025750A002A2A2A204E20636D642073796E746178206572726F720A002A2A2A2038
:203DEE00556E6B6E6F776E20636F6D6D616E643A205B25735D0A0054305469636B7320254B
:203E0E00750A004553455400436861722064656C61792069732025752078203130302075A3
:203E2E00730A002A2A2A205420636F6D6D616E6420737472696E67206973206D697373690E
:203E4E006E670A00417661696C61626C6520636F6D6D616E6473202876616C756573206921
:203E6E006E20646563696D616C20756E6C657373206E6F746564290A0020413D7374726950
:203E8E006E672020202B20736574206E6574776F726B206164647265737320746F2073740E
:203EAE0072696E670A002044202020202020202020202A20646973706C617920696E746586
:203ECE00726E616C20737461747573207661726961626C65732028736F6D6520696E20680F
:203EEE006578290A002045202020202020202020202A2073686F7720616E6420636C6561EC
:203F0E0072206572726F7220666C6167730A00204C206E202020202020202020207365741A
:203F2E00207265706F7274696E67206D6F646520286269746D6170706564290A00204E20F5
:203F4E006E202020202020202A2B20736574206E6574776F726B206D6F64650A00205120BA
:203F6E002020202020202020202020717565727920696E707574730A00205245534554200D
:203F8E0020202020202020706572666F726D20706F7765722D6F6E20726573657420696EA7
:203FAE00697469616C697A6174696F6E0A002052206E20202020202020202020736574202C
:203FCE006368617261637465722064656C617920666F72205420636F6D6D616E640A0020F3
:203FEE0053202020202020202020202020736574206F75747075740A0020542020202020A5
:20400E002020202020202073656E64204153434949207465787420737472696E670A002BAE
:20402E00206D61726B73206E6574776F726B2D6F6E6C7920636F6D6D616E64730A002A2055
:20404E006D61726B7320646562756767696E6720636F6D6D616E64730A00577269746520C1
:20406E002530327820746F206164647265737320253034780A005265616420253032782044
:20408E0066726F6D206164647265737320253034782025730A0066616B65640000496E695A
:2040AE007469616C697A696E672064657669636520696E666F726D6174696F6E0A00202E79
:2040CE002E2E25733A20002072656164790A002A2A2A2042616420646576696365206E6121
:2040EE006D65205B25735D0A005B446576696365202573002C20626974204944203D202529
:20410E00755D0A000A2A2A2A20426164206269742049443A2025750A005D0A002A2A2A20F7
:20412E0053657420636F6D6D616E64206D697373696E6720646174610A002A2A2A204D6914
:20414E007373696E67206368616E6E656C0A002A2A2A204269742076616C7565206D7573BB
:20416E00742062652030206F7220310A002A2A2A20446576696365202573206E6F7420698A
:20418E006E7374616C6C65640A002A2A2A2043616E6E6F74207365742076616C75650A00FC
:2041AE002A2A2A20426164206465766963650A002E2575003D0025750025303478002530BD
:2041CE003278002575001B000C000A000D000A44494F2D4C696E6B204E6574776F726B653F
:2041EE0064204469676974616C20492F4F2C2056657273696F6E2000312E3067000A2020F6
:20420E00436F70797269676874203139393220436972637569742043656C6C61722C2049E7
:1F422E006E632E0A002D2D2D2046656C6C206F75742074686520626F74746F6D210A0085
:00000001FF
